:020000040000FA
:10000000905A0020C1010000C9010000CB0100008E
:10001000CD010000CF010000D10100000000000070
:10002000000000000000000000000000D3010000FC
:10003000D501000000000000D70100009902000077
:10004000DB010000DD010000DF010000E101000034
:10005000E3010000E5010000E7010000E901000004
:10006000EB010000ED010000EF010000F1010000D4
:10007000F3010000F5010000F7010000F9010000A4
:10008000C1080000FD010000FF01000001020000A6
:100090000302000005020000070200000902000040
:1000A0000B0200000D0200000F0200001102000010
:1000B00013020000150200001702000019020000E0
:1000C0001B0200001D0200001F02000021020000B0
:1000D000230200007518000027020000290200001A
:1000E0002B0200002D0200002F0200003102000050
:1000F0003302000035020000370200003902000020
:100100003B0200003D0200003F02000041020000EF
:1001100043020000450200004702000049020000BF
:100120004B0200004D0200004F020000510200008F
:10013000530200005502000057020000590200005F
:100140005B0200005D0200005F020000610200002F
:1001500063020000650200006702000069020000FF
:100160006B0200006D0200006F02000071020000CF
:10017000730200007502000005090000790200000A
:100180007B0200007D0200007F020000810200006F
:10019000830200008502000087020000890200003F
:1001A0008B0200008D020000DFF810D000F054FB3D
:1001B00000F0D6F80048004715320000905A0020A1
:1001C0003348804733480047FEE7FEE7FEE7FEE797
:1001D000FEE7FEE7FEE7FEE7FEE7FEE7FEE7FEE7F7
:1001E000FEE7FEE7FEE7FEE7FEE7FEE7FEE7FEE7E7
:1001F000FEE7FEE7FEE7FEE7FEE7FEE7FEE7FEE7D7
:10020000FEE7FEE7FEE7FEE7FEE7FEE7FEE7FEE7C6
:10021000FEE7FEE7FEE7FEE7FEE7FEE7FEE7FEE7B6
:10022000FEE7FEE7FEE7FEE7FEE7FEE7FEE7FEE7A6
:10023000FEE7FEE7FEE7FEE7FEE7FEE7FEE7FEE796
:10024000FEE7FEE7FEE7FEE7FEE7FEE7FEE7FEE786
:10025000FEE7FEE7FEE7FEE7FEE7FEE7FEE7FEE776
:10026000FEE7FEE7FEE7FEE7FEE7FEE7FEE7FEE766
:10027000FEE7FEE7FEE7FEE7FEE7FEE7FEE7FEE756
:10028000FEE7FEE7FEE7FEE7FEE7FEE7FEE700002B
:100290008D170000A901000030B410B50348804755
:1002A00030BCAE4630BC0248004770471D340000E9
:1002B000512500002DE9F0410024061B254671F16F
:1002C000000605DA01240027D0EB070067EB0101E7
:1002D000161E73F1000605DA0027D2EB070201258E
:1002E00067EB030300F0D1F886460E4617469C469E
:1002F000AC4204D00025D0EB050E65EB010624B11D
:100300000020D2EB000760EB030C704631463A4602
:100310006346BDE8F08140EA01039B0703D009E092
:1003200008C9121F08C0042AFAD203E011F8013BE1
:1003300000F8013B521EF9D27047D2B201E000F83A
:10034000012B491EFBD270470022F6E710B5134679
:100350000A4604461946FFF7F0FF204610BD00008C
:1003600070B5054C054D04E02046016808448047FF
:10037000241DAC42F8D170BDF83F0000FC3F0000E6
:100380002DE9F04D81EA030404F0004B21F0004513
:1003900014464FF0000A23F0004150EA050220D035
:1003A00054EA01021DD0C5F30A570246C5F31303F0
:1003B000C1F31300C1F30A5640F4801543F48013CF
:1003C000A7EB0608101BD64608F2FD3873EB0500B4
:1003D00002D308F1010801E092185B41B8F1000F67
:1003E00003DA00200146BDE8F08D00204FF48011B3
:1003F000064684460EE0171B73EB050705D3121B58
:1004000063EB050306434CEA010C49084FEA300050
:1004100092185B4150EA0107EDD152EA030012D075
:1004200082EA040083EA0501084305D0101BAB41B2
:1004300006D20122002306E000224FF0004302E032
:100440006FF0010253101AEB06004CEB085110EB51
:100450000A0041EB0B01BDE8F04D00F057B830B594
:100460000B46014600202022012409E021FA02F572
:100470009D4205D303FA02F5491B04FA02F528440C
:10048000151EA2F10102F1DC30BD2DE9F05F054639
:10049000002092469B4688460646814640241BE043
:1004A000284641464746224600F020F853465A4621
:1004B000C01A914110D311461846224600F0DEF9C9
:1004C0002D1A67EB01084F4622460120002100F05B
:1004D000D5F917EB00094E41201EA4F10104DFDC21
:1004E000484631462A464346BDE8F09F202A04DBB1
:1004F000203A21FA02F00021704721FA02F3D0409D
:10050000C2F12002914008431946704710B5141EED
:1005100073F1000408DA401C41F1000192185B41BC
:100520001A4301D120F0010010BD2DE9F04D924693
:100530009B4611B1B1FA81F202E0B0FA80F22032AA
:10054000904600F09BF904460F4640EA0A0041EA53
:100550000B0153465A46084313D0114653EA010093
:1005600019D0C8F140025046FFF7C0FF05460E46BD
:1005700050465946424600F081F9084305D0012013
:1005800004E020463946BDE8F08D0020054346EAE8
:10059000E0762C4337430A986305E40AA0EB080091
:1005A0000022FD0A44EA47540A3002D500200146E1
:1005B000E9E7010510196941DDE9084500196941BC
:1005C000BDE8F04DA2E72DE9FE4F804681EA030029
:1005D000C00F0C46009021F0004123F00045B8EB1D
:1005E0000200A94105D24046214690461C460B46D2
:1005F000024623F00040104347D0270DC7F30A00FE
:10060000C3F30A510290401A019040286BDAC3F3F9
:10061000130040F4801B0098924620B10023D2EBD7
:10062000030A63EB0B0B01985946C0F14002504698
:1006300000F024F906460D4650465946019A00F04E
:100640002CF910EB08006141002487EA115284EA7A
:10065000E7731A4340D0009A62B3019A012A4FEA25
:10066000075215DC001B61EB02014FF0004202EA69
:100670000752CDE90042001C41F5801132462B465D
:10068000FFF753FF03B0BDE8F08F40462146F9E77E
:10069000001B61EB0201001C41F5801300185B4157
:1006A0002018A2F5001747EB030140EAD570B619F0
:1006B0006D4111E06D084FEA360645EAC0754FEA14
:1006C0000752001B61EB0201001C41F58011490833
:1006D0004FEA30000019514132462B4603B0BDE8C5
:1006E000F04FFFF713BF0098012240000023D0EB2A
:1006F000020263EBE073009821464FEAE074B8EB26
:10070000000061EB0401E9E783F000435BE781F05F
:10071000004158E72DE9FE4F81EA030404F000444C
:1007200021F0004100944FF0000B23F0004350EA09
:1007300001045ED052EA03045BD0C3F30A54C1F350
:100740000A552C44A4F2F3340194A0FB0254C1F3E3
:10075000130141F48011C3F3130343F4801301FB2D
:10076000024400FB034E840A970A44EA815447EA94
:100770008357A4FB076802958D0A05FB07854FEA9E
:10078000932C04FB0C542705029D4FEA065847EAB8
:100790001637B5EB08056EEB070C870E920E47EA8D
:1007A000811742EA8312A7FB0201B6EB0B0164EB4F
:1007B00000042B0D43EA0C335E1844EB1C50DA4660
:1007C0005146E7FB0201C5F313044FEA0B3343EA3A
:1007D00014534FEA0432019C43EA0603A4F10C04CB
:1007E0000294009CCDE900B4FFF79FFE03B0BDE882
:1007F000F08F00200146F9E7C1F30A52C1F313015B
:1008000040F2FF3341F480119A4202DA002001469F
:10081000704740F233439A42A2F2334202DC524222
:10082000FFF764BE00F02AB830B5041E71F1000471
:1008300004DB4FF00044404264EB0101141E73F1ED
:10084000000405DB1C464FF00043524263EB0403F7
:10085000994208BF904230BD064C074D06E0E06863
:1008600040F0010394E8070098471034AC42F6D3F7
:10087000FFF79EFCD83F0000F83F0000202A04DB71
:10088000203A00FA02F1002070479140C2F12003A3
:1008900020FA03F3194390407047202A06DBCB1758
:1008A000203A41FA02F043EAE07306E041FA02F32B
:1008B000D040C2F120029140084319467047000021
:1008C00080B582B048F20000C4F20A0000F03CF8A3
:1008D00001909DF80400C00788B1FFE741F2701154
:1008E000C2F2000148F20000C4F20A0000F032F83F
:1008F00040F28801C2F2000101200870FFE702B057
:1009000080BD000080B582B048F60000C4F20A0045
:1009100000F01AF801909DF80400C00788B1FFE7C5
:1009200041F28011C2F2000148F60000C4F20A0050
:1009300000F010F840F28901C2F2000101200870B5
:10094000FFE702B080BD000081B000900098C06851
:1009500001B0704783B0029001910298006CC0B260
:10096000C009019908710298006CC0F380100199C8
:1009700048710298006C00F00F000199887101988D
:10098000007908BBFFE70298406CC0000299896CAF
:1009900040EA51100199086000200090FFE700989C
:1009A0000199897988420ED2FFE70298009900EBFD
:1009B0008100C06C0199009A1144C871FFE700984A
:1009C00001300090EBE728E00298406C4005029966
:1009D000896C40EA41300299C96C40EA41100299A1
:1009E000096D40EAD1000199086000200090FFE7FE
:1009F00000980199897988420ED2FFE70298009900
:100A000000EB8100406D0199009A1144C871FFE725
:100A1000009801300090EBE7FFE70299042048605E
:100A200003B0704780B582B08DF80700062002F051
:100A3000ABFD9DF8070002F0B9FD02F097FD8DF8BF
:100A4000060002F043FD43F6C470C0F2000002F05D
:100A5000B7FD9DF8061043F68D70C0F2000002F05D
:100A6000AFFD9DF8060002B080BD000080B582B0E9
:100A7000292002F089FD022002F080FA02F076FDC2
:100A80008DF8070002F022FD9DF8070002B080BD3E
:100A900080B582B0262002F077FD02F067FD8DF868
:100AA000070002F013FD9DF8070002B080BD0000B2
:100AB00080B582B00190282002F066FD00208DF8FC
:100AC0000300FFE79DF8030007280DDCFFE702F0B5
:100AD0004DFD01994A1C01920870FFE79DF8030043
:100AE00001308DF80300EDE702F0F0FC02B080BDAC
:100AF00080B582B000208DF80700012002F044FD8F
:100B000002F034FD8DF8070002F0E0FC9DF80700CC
:100B100002B080BD80B582B000208DF806008DF84F
:100B20000500272002F030FD02F0D0FCFFE70A208C
:100B300002F0DAF943F6B270C0F2000002F040FDB4
:100B40009DF8051043F68D70C0F2000002F038FDEC
:100B500000F086F88DF805009DF80500102801D0FA
:100B6000FFE70CE09DF80600411C8DF80610C9282F
:100B700004DBFFE7FA208DF8070005E0D7E79DF8D2
:100B800005008DF80700FFE79DF8070002B080BD63
:100B900080B5052002F0F8FC02F098FC80BD000052
:100BA00080B582B00190232002F0EEFC00208DF889
:100BB0000300FFE79DF8030003280DDCFFE7019821
:100BC000411C0191007802F0F1FCFFE79DF8030061
:100BD00001308DF80300EDE702F078FC02B080BD33
:100BE00080B582B00190222002F0CEFC00208DF86A
:100BF0000300FFE79DF8030003280DDCFFE70198E1
:100C0000411C0191007802F0D1FCFFE79DF8030040
:100C100001308DF80300EDE702F058FC02B080BD12
:100C200080B582B00190242002F0AEFC00208DF847
:100C30000300FFE79DF8030003280DDCFFE70198A0
:100C4000411C0191007802F0B1FCFFE79DF8030020
:100C500001308DF80300EDE702F038FC02B080BDF2
:100C600080B582B02C2002F08FFC02F07FFC8DF862
:100C7000070002F02BFC9DF8070002B080BD0000C9
:100C800080B584B08DF80F00ADF80C100292BDF85D
:100C90000C0008B9FFE72DE03C2002F075FC9DF840
:100CA0000F0002F083FC9DF80C0002F07FFC9DF821
:100CB0000D0002F07BFC012002F060F90020ADF88D
:100CC0000600FFE7BDF80600BDF80C1088420EDAFA
:100CD000FFE702F04BFC0299087002980130029085
:100CE000FFE7BDF806000130ADF80600EAE702F0C4
:100CF000EDFBFFE704B080BD80B582B08DF8070042
:100D00003B2002F041FC9DF8070002F04FFC02F08E
:100D10002DFCADF8040002F029FC0146BDF80400EA
:100D200000EB0120ADF8040002F0D0FBBDF8040098
:100D300002B080BD80B582B08DF80700302002F08F
:100D400023FC9DF8070002F031FC022002F016F9A6
:100D500002F00CFC8DF8060002F0B8FB9DF80600CE
:100D600002B080BD80B584B0FFF780FEADF80E0004
:100D70009DF80E00C00720B1FFE701A8FFF798FE1D
:100D8000FFE7BDF80E008007002801D5FFE7FFE769
:100D9000BDF80E004007002807D5FFE743F6F160D5
:100DA000C0F2000002F00CFCFFE7BDF80E00C00628
:100DB000002804D5FFE7002000F042F9FFE7BDF866
:100DC0000E008006002804D5FFE7012000F038F966
:100DD000FFE7BDF80E004006002804D5FFE702201B
:100DE00000F02EF9FFE7BDF80E000006002804D53C
:100DF000FFE7032000F024F9FFE704B080BD000006
:100E000080B584B06520FFF70DFE8DF80E009DF8CB
:100E10000E009A2804D0FFE7FA208DF80F0030E08A
:100E200043F6A870C0F20000019002F0C9FB9DF8E3
:100E30000E1043F68D70C0F20000029002F0C0FB6D
:100E400040F28C00C2F200000090FFF7C9FE00984B
:100E50000430FFF7A5FE00980830FFF7E1FEFFF72A
:100E600059FE014601988DF80E1002F0A9FB029878
:100E70009DF80E1002F0A4FB9DF80E008DF80F00F7
:100E8000FFE79DF80F0004B080BD000080B582B080
:100E90008DF8060000208DF805008DF8040035203F
:100EA00002F072FB9DF8060002F080FB02F00EFBE0
:100EB000FFE7052002F018F8FFF7D2FE8DF80400D6
:100EC0009DF80400102801D0FFE70CE09DF8050014
:100ED000411C8DF80510C92804DBFFE7FA208DF8C6
:100EE000070005E0E5E79DF804008DF80700FFE73F
:100EF0009DF8070002B080BD80B584B08DF80F006A
:100F00000291ADF80620392002F03EFB9DF80F005B
:100F100002F04CFB9DF8060002F048FB9DF807002C
:100F200002F044FB0020ADF80400FFE7BDF8040028
:100F3000BDF8061088420DDAFFE70298411C0291C5
:100F4000007802F033FBFFE7BDF804000130ADF894
:100F50000400EBE702F0BAFA04B080BD80B582B0BD
:100F60008DF807000091312002F00EFB9DF807007C
:100F700002F01CFB0098411C0091007802F016FB67
:100F80000098411C0091007802F010FB0098411C71
:100F90000091007802F00AFB0098411C0091007853
:100FA00002F004FB02F092FA02B080BD80B582B07C
:100FB0008DF80700ADF80410322002F0E5FA9DF834
:100FC000070002F0F3FA9DF8040002F0EFFA9DF832
:100FD000050002F0EBFA02F079FA02B080BD0000E1
:100FE00080B582B08DF807008DF80610342002F02D
:100FF000CBFA9DF8070002F0D9FA9DF8060002F03E
:10100000D5FA02F063FA02B080BD000080B582B06C
:101010008DF80700ADF80410332002F0B5FA9DF802
:10102000070002F0C3FA9DF8040002F0BFFA9DF831
:10103000050002F0BBFA02F049FA02B080BD0000E0
:1010400080B582B08DF807009DF80700FFF772FEAB
:101050008DF806009DF80600C00708B1FFE7FFE71E
:101060009DF806008007002801D5FFE7FFE79DF8FF
:1010700006004007002825D5FFE79DF80700FFF789
:101080003BFEADF80400BDF8041043F64C70C0F20E
:10109000000002F095FA9DF80700BDF8041040F238
:1010A000B002C2F20002009202EB0032FFF7E8FD4C
:1010B00000999DF8070001EB0031BDF80420FFF70F
:1010C0001BFFFFE79DF806000007002807D5FFE794
:1010D00043F61670C0F2000002F072FAFFE79DF8C6
:1010E0000600C006002807D5FFE743F6D960C0F226
:1010F000000002F065FAFFE79DF8060040060028B0
:1011000007D5FFE743F62A70C0F2000002F058FA54
:10111000FFE702B080BD000080B582B001900020E2
:101120008DF80300019844F60001C4F204018842DE
:1011300009D1FFE7019840F24801C2F200010860BE
:1011400001F024F8FFE7019844F20001C4F2040121
:10115000884209D1FFE7019840F24801C2F200013C
:10116000086000F095FFFFE700F05CFF8DF80300DA
:1011700002B080BD82B001900091009901208840AA
:101180000199086202B0704782B001900091009905
:10119000012000FA01F2019948691043486102B048
:1011A0007047000082B0019000910198C0690099D9
:1011B000C84000F0010002B07047000082B001900A
:1011C00041F64020C2F20000007818B9FFE7002085
:1011D00000900EE00199C1F3C62241F6C010C2F2A0
:1011E0000000805CC1F30221C84000F001000090C3
:1011F000FFE7009802B0704780B584B0FFE741F682
:101200004020C2F200008069029000F0B9FA039019
:101210000398029988420FD2FFE700F059FE50B9B7
:10122000FFE741F64021C2F2000108690130086180
:1012300001F03EFCFFE7FFE7039801F043FC01905B
:10124000FFE7029801998842D9D1FFE7039804B0DB
:1012500080BD000080B58CB0099008910792089875
:1012600028B1FFE70798B0F5807F03D9FFE700209A
:101270000A90AFE00998FFF7A1FF18B9FFE7012036
:101280000A90A7E0FFF7B8FF0590BDF82400099089
:10129000EFF305800B900B9A099840F40021002A87
:1012A00018BF0846099008980690079850B9FFE7BC
:1012B0000998059900231A4600F090F801900198CA
:1012C0000A9087E0079808281BD8FFE700200290C3
:1012D00003900699079A02A8FFF71DF8079800F0F7
:1012E0000701099840EA01400990099840F04070D0
:1012F0000599029A039B00F071F8019001980A90F9
:1013000068E000F02FFC01464FF4E02000EA0140C5
:10131000049006990868496803910290069808307D
:10132000069007980838079004990998084309908F
:10133000099840F080700599029A039B00F04EF8DE
:101340000190019818B9FFE700200A9042E0049844
:101350004FF6017108430990FFE7079809281CD34D
:10136000FFE70699086849680391029006980830DB
:10137000069007980838079009980599029A039BE8
:1013800000F02CF80190099801300990019818B9E3
:10139000FFE700200A901DE0DFE7002002900390A5
:1013A0000699079A02A8FEF7B6FF099820F47F4035
:1013B00009900799099840EA01200990099840F09E
:1013C00000700599029A039B00F008F801900198BB
:1013D0000A90FFE70A980CB080BD000080B58CB081
:1013E0000A9009910892079307200590FFE7059856
:1013F00000286AD0FFE700F0BFFB0490049800F0DB
:101400007F0141F2C010C2F2000000EB0110069013
:1014100004994FF4700000EA413001900A98019954
:101420000843099A4FF0805101EAD2010843089A13
:101430004FF0005101EA92010843079A4FF08041B2
:1014400001EA5201084340F04060039006980C30D6
:10145000039900F021FD03909DF80F00400700283C
:101460002ED5FFE7039880F080600390039880F00A
:1014700000400390039800F000400290099820F08B
:1014800000400299084306990860089820F000403F
:101490000299084306994860079820F00040029995
:1014A00008430699886006980C30039901F0E6FA23
:1014B00028B1FFE700F074FB01200B900AE004E084
:1014C000FFE705980138059091E700F05FFB0020E9
:1014D0000B90FFE70B980CB080BD000087B0059023
:1014E000049103920498FE2804D8FFE70398FF288C
:1014F00003D3FFE70020069036E000200290019021
:10150000FFE7019803282CD8FFE705980199C84008
:10151000C007F0B1FFE704980090FFE70098039937
:10152000884215D8FFE7009901F00702012000FA70
:1015300002F3029800EBD10241F6C011C2F20001A1
:10154000885C18438854FFE7009801300090E5E775
:10155000FFE7029820300290FFE7019801300190E8
:10156000CFE701200690FFE7069807B0704700001C
:1015700080B58AB00990089141F64021C2F200017D
:1015800001910020087041F6C010C2F200008021D5
:10159000FEF7DAFE43F6B460C0F20000182101F055
:1015A00025FC01460198ADF81A10006A42F26B71F1
:1015B000CEF2A51188420FD0FFE741F64021C2F2DA
:1015C000000142F26B70CEF2A5100862BDF81A005D
:1015D00048800120C8611CE041F64020C2F20000B2
:1015E0004088BDF81A1088420AD0FFE7BDF81A00FB
:1015F00041F64021C2F2000148800120C86107E0A5
:1016000041F64021C2F20001C8690130C861FFE71C
:10161000FFE741F64020C2F20000C069012812D164
:10162000FFE741F64021C2F2000100204870486007
:101630008860C86041F2C010C2F200004FF400613F
:10164000FEF782FE20E000200290FFE702987F284C
:1016500019D8FFE7029941F2C010C2F2000000EB76
:10166000011007900798C07B4007002806D5FFE7C8
:101670000799C86820F04060C860FFE7FFE702985C
:1016800001300290E2E7FFE741F64020C2F200009D
:10169000C06901281CD1FFE700F076F80490049897
:1016A00020B1FFE74FF47A70059002E0002005902A
:1016B000FFE7059841F64021C2F200014861002091
:1016C0008861086141F2D801C2F20001087003E0AC
:1016D00000F05AF80490FFE7049838B3FFE7099840
:1016E0000021FE220092FFF7F9FE0F20EF221146A3
:1016F000FFF7F4FE009A04201146FFF7EFFEFFF714
:101700007BFD0390039941F64020C2F2000043693B
:10171000C2694FF60070C0F20030FFF75FFE089814
:1017200018B1FFE700F006F8FFE7FFE704980AB0FA
:1017300080BD000080B584B041F64020C2F20000B8
:10174000007818B1FFE70120039015E041F6402131
:10175000C2F20001012001900870FFF74DFD0290D8
:1017600002994FF60170C0F2003000231A46FFF7CD
:1017700035FE01980390FFE7039804B080BD000098
:1017800080B501F099FC80BD012070474EF688516C
:10179000CEF20001086840F4700008607047000055
:1017A00080B584B00290EFF3108072B60390029877
:1017B00001901E2810D0FFE7019828281AD0FFE7D3
:1017C0000198502824D0FFE7019878282ED0FFE711
:1017D000019896283AD03AE048F6491040F6A171AF
:1017E0004FF6AC72C0F6113240F23143C1F2001331
:1017F00098473CE048F6492041F2A9414FF6AC72C7
:10180000C0F6113240F23143C1F2001398472EE086
:101810004DF2493042F64A114FF6AC72C0F6113221
:1018200040F23143C1F20013984720E041F689406D
:10183000C0F2010043F66B514FF6AC72C0F61132A4
:1018400040F23143C1F20013984710E0FFE746F23F
:101850008950C0F2010044F674414FF6AC72C0F6F4
:10186000113240F23143C1F200139847FFE762B6EC
:1018700004B080BD80B582B00020019040F24800E5
:10188000C2F20000006844F20001C4F20401884280
:1018900014D1FFE741F20000C4F204000C21FFF76D
:1018A00081FC50B1FFE741F20000C4F204000C21BA
:1018B000FFF760FC01200190FFE7FFE740F24800DE
:1018C000C2F20000006844F60001C4F2040188423C
:1018D00014D1FFE741F20000C4F204000D21FFF72C
:1018E00061FC50B1FFE741F20000C4F204000D2199
:1018F000FFF740FC01200190FFE7FFE7019818B1D6
:10190000FFE7FFF72FFAFFE702B080BD82B001903A
:1019100000910099012000FA01F2019908689043B2
:10192000086002B07047000082B0019000910198F9
:10193000006B0099C84000F0010002B07047000041
:1019400080B586B0DDF824C0DDF820C00590049194
:10195000039202930020C4F20A00019005980090BF
:10196000B0F1402F6BD0FFE7009844F60001C4F2BD
:10197000000188426FD0FFE700980021C4F2040103
:10198000884220D0FFE7009840F60001C4F204012D
:10199000884224D0FFE7009841F20001C4F204011C
:1019A000884228D0FFE7009841F60001C4F2040104
:1019B00088422CD0FFE7009841F20001C4F20A01EE
:1019C000884230D053E00821C4F20001086840F09A
:1019D000010008600020C4F20A00019047E00821DD
:1019E000C4F20001086840F0020008601020C4F250
:1019F0000A0001903BE00821C4F20001086840F0B1
:101A0000040008602020C4F20A0001902FE00821A1
:101A1000C4F20001086840F0080008603020C4F2F9
:101A20000A00019023E00C21C4F20001086840F094
:101A3000010008604020C4F20A00019017E008216C
:101A4000C4F20001086840F0100008608020C4F271
:101A50000A0001900BE00821C4F20001086840F080
:101A6000200008609020C4F20A000190FFE701986E
:101A700004990022012300F087FA0398012809D174
:101A8000FFE70499012000FA01F205994868104324
:101A9000486008E00499012000FA01F205994868BD
:101AA00090434860FFE7029801280BD1FFE70499B3
:101AB000012000FA01F20199D1F800011043C1F8A8
:101AC00000010AE00499012000FA01F20199D1F81D
:101AD00000019043C1F80001FFE7089801280BD1ED
:101AE000FFE70499012000FA01F20199D1F8000200
:101AF0001043C1F800020AE00499012000FA01F243
:101B00000199D1F800029043C1F80002FFE709985B
:101B100001280BD1FFE70499012000FA01F2019995
:101B2000D1F800041043C1F800040AE00499012030
:101B300000FA01F20199D1F800049043C1F80004C1
:101B4000FFE706B080BD000082B0019000910099CF
:101B5000012000FA01F2019908681043086002B000
:101B60007047000080B541F64020C2F2000001300D
:101B700001F0D8F880BD000080B541F64020C2F2E7
:101B80000000043001F0BEF880BD000080B541F6D1
:101B90004020C2F200000C3001F0B4F880BD00001B
:101BA00080B541F64020C2F20000083001F0AAF8EA
:101BB00080BD000080B582B040F28C00C2F200000F
:101BC00001902421FEF7C0FB01994AF6C000C0F63F
:101BD0003D2008604AF6C000C0F23D1048606FF03A
:101BE0007F40886002B080BD80B584B000208DF851
:101BF0000F000290FFE70298002866DCFFE70298DA
:101C000041F2B401C2F20001019101EB4012430123
:101C100000200090C850D061906150611061D06088
:101C2000906050600298430100EB800240F2540043
:101C3000C2F2000050F81220CA50029B03EB83024C
:101C400000EB4202D28801EB43139A82029B03EB22
:101C5000830200EB4202928801EB4313DA82029A7C
:101C600002EB820300EB4300007A01EB4212907218
:101C7000029801EB4011C0B2FFF770F90199029888
:101C800001EB4011897AC0B2FFF7AAF901990298D5
:101C900001EB4011898AC0B2FFF788F901990298D7
:101CA00001EB4011C98AC0B2FFF7B0F99DF80800F6
:101CB000FFF7ECF88DF80F009DF80F0001F08EFA99
:101CC000FFE702980130029095E704B080BD000064
:101CD00080B586B040F24800C2F20000006844F2CD
:101CE0000001C4F20401884213D1FFE768460022D4
:101CF0004260026041F20000C4F2040004900C2132
:101D000005910123FFF71CFE04980599FFF73CFAA3
:101D1000FFE740F24800C2F20000006844F600010C
:101D2000C4F20401884213D1FFE7684600224260F2
:101D3000026041F20000C4F2040002900D21039100
:101D40000123FFF7FDFD02980399FFF71DFAFFE756
:101D5000252000F095FF06B080BD000080B582B060
:101D6000684600234360036041F60000C4F20400AB
:101D700009210122FFF7E4FD02B080BD80B582B0E9
:101D800044F60000C4F20400019000208DF8030026
:101D90000198FFF7C1F9FFF79BFFFEF7F9FE6420FA
:101DA00001F0A2F843F65F70C0F2000001F008FCF9
:101DB000FEF79EFE8DF803009DF8031043F6977022
:101DC000C0F2000001F0FCFB322001F08DF8FFF7BB
:101DD000F1FEFFF715F88DF803009DF8030001F000
:101DE000FDF9FFE7FEF754FE012804D1FFE7C82004
:101DF00001F07AF806E043F67470C0F2000001F0DA
:101E0000DFFB00E0EEE7FFF7EFFE02B080BD000071
:101E100080B582B0019040F20800C2F20000006874
:101E20000199B0FBF1F000F045FB02B080BD00006D
:101E300080B500F029F842F65520C0F2000000F00D
:101E40002FFBFFF78BFF4FF47A70FFF7E1FF0120C4
:101E500001F07CF943F6CC60C0F2000001F0B0FB69
:101E600080BD000080B582B040F60000C4F20A00D8
:101E7000019000214FF4806200F03AFE019800F0DA
:101E800083FE02B080BD000080B50F200121FFF766
:101E90006FFBFFF74FFC80BD10B585B00490039138
:101EA000049B039C53E8002F900103D3BFF32F8FB3
:101EB000002206E002F00042224343E8002101B183
:101EC000F0E7029201910090029805B010BD000069
:101ED00080B541F2D800C2F20000012100F044FFB9
:101EE00080BD000080B584B00020C4F20A000190DB
:101EF00003210F2202920023039300F045F801987A
:101F0000029A039B042100F03FF84AF22001C4F238
:101F10000A0108682222C0F20F021043086000F094
:101F2000A7FF00F0A5FF4AF24001C4F20A010868C9
:101F300020F0020008604AF24402C4F20A0210686B
:101F40004FF60063CFF6E0431840106010683C2362
:101F5000C0F2030318431060086820F00400086012
:101F6000FFE74AF24C00C4F20A00006808B9FFE734
:101F7000F7E74AF24001C4F20A01086840F00100A4
:101F8000086004B080BD000084B00390029101920B
:101F900000930298072813D8FFE7029881000F20CA
:101FA00000FA01F2039908689043086001980299C9
:101FB000890000FA01F2039908681043086016E0EE
:101FC00002986FF01F0101EB80020F2000FA02F36C
:101FD000039A5068984350600198029A01EB82017D
:101FE00000FA01F20399486810434860FFE700983F
:101FF00058B1FFE70299012000FA01F20399D1F8E4
:1020000000031043C1F800030AE00299012000FA1E
:1020100001F20399D1F800039043C1F80003FFE7F0
:1020200004B0704780B582B000208DF8070040F200
:102030004800C2F20000006844F60001C4F2040146
:1020400088420AD1FFE741F20000C4F204000D21EA
:10205000FFF76AFC8DF80700FFE740F24800C2F284
:102060000000006844F20001C4F2040188420AD171
:10207000FFE741F20000C4F204000C21FFF754FC1A
:102080008DF80700FFE79DF8070002B080BD000053
:1020900080B58EB06846002209924260026041F22B
:1020A0000000C4F204000C2101230893FFF748FC50
:1020B000089A099B68464360036040F60000C4F23A
:1020C000040002900E210391FFF73AFC0298039955
:1020D000FFF71CFC4FF4967000F006FF029803997E
:1020E000FFF732FD4FF04020049003210791FFF7E6
:1020F0002BFD04980799089A099BEC46CCF804300C
:10210000CCF80030FFF71CFC04980799FFF71CFD82
:10211000089A099B8020C4F20A00059002210691CA
:10212000FFF732FF0598089B04211A46FFF72CFFA2
:102130000598069A099B0521FFF726FF079A08993B
:1021400009988DF831208DF82C008DF82D108DF820
:102150002E1008228DF82F208DF830108DF83200C7
:102160008DF833008DF834008DF835008DF8360089
:1021700044F20000C4F204000A900BA900F08CF8AD
:102180000A9800F071F90EB080BD000080B58CB0E7
:102190006846002207924260026041F20000C4F2E9
:1021A00004000D2101230693FFF7CAFB069A079B43
:1021B00068464360036040F60000C4F204000290E9
:1021C0000C210391FFF7BCFB02980399FFF79EFBDC
:1021D0004FF4967000F088FE02980399FFF7B4FC64
:1021E000069944F60000C4F200000490FFF7ACFC2E
:1021F0000498069A079B69464B600B601146FFF7EF
:102200009FFB04980699FFF79FFC069A079B902076
:10221000C4F20A0005901946FFF7B6FE0598069B22
:1022200004211A46FFF7B0FE0598079B05210222FC
:10223000FFF7AAFE0699079803228DF829208DF84A
:1022400024008DF825108DF8261008228DF82720FF
:102250008DF828108DF82A008DF82B008DF82C00B1
:102260008DF82D008DF82E0044F60000C4F2040015
:10227000089009A900F010F8089800F0F5F80CB0E3
:1022800080BD000081B000900099086820F008002F
:10229000086001B07047000080B588B007900691D3
:1022A0000020059004900798039044F20001C4F2C6
:1022B0000401884208D0FFE7039844F60001C4F205
:1022C0000401884208D00FE00821C4F20001086828
:1022D00040F40050086007E00821C4F200010868DB
:1022E00040F480400860FFE70798FFF7CBFF0698AF
:1022F0004079082804D1FFE701200590049007E009
:102300000698407918B9FFE701200490FFE7FFE73E
:10231000079908684EF20802CFF601721040086073
:102320000698017890F801C08278C378890241EA62
:102330000C2141EA42216FF00F0202EB031211431C
:10234000027941EA0231059A41EA4231049A41EAAE
:102350004271427902F0070211430291807901280B
:1023600005DBFFE7069880790138019002E0002044
:102370000190FFE70298019940EA81400699097AA5
:1023800040EA415007990A68104340F040700860E5
:102390000799086820F040700860079940F27F3084
:1023A000086107990020C8600699C8794A7A897A35
:1023B000400140EA821040EA41220799C868104370
:1023C000C8600798009044F20001C4F204018842FA
:1023D00008D0FFE7009844F60001C4F204018842E7
:1023E00011D021E00699C8794A7A897A10430843C6
:1023F00020B1FFE7052000F013FC03E0052000F00A
:10240000D7FBFFE710E00699C8794A7A897A10432A
:10241000084320B1FFE7112000F002FC03E0112087
:1024200000F0C6FBFFE7FFE708B080BD80B540F2D3
:102430004800C2F200000068002100F01FF8C0B29E
:1024400080BD000080B582B08DF8070040F24800E2
:10245000C2F2000000689DF8071000F00FF88DF838
:10246000060002B080BD000081B0009000990868AD
:1024700040F00800086001B07047000082B0019091
:102480000091009801994860FFE701988068000773
:10249000002801D4FFE7F8E70198406802B07047D0
:1024A00081B00090009841F2B001C2F200010860D2
:1024B00001B0704780B584B0029002980138B0F145
:1024C000807F03D3FFE7012003901AE002980138D0
:1024D0004EF21401CEF2000108604FF0FF300721E8
:1024E000019100F0E5FB01994EF21802CEF20002D4
:1024F000002010604EF21002CEF200021160039034
:10250000FFE7039804B080BD82B0009000980138C6
:10251000B0F1807F03D3FFE70120019015E04EF278
:102520001002CEF2000200201060009901394EF234
:102530001403CEF2000319604EF21801CEF200012E
:102540000860072111600190FFE7019802B0704711
:1025500080B541F2B000C2F20000006838B1FFE778
:1025600041F2B000C2F2000000688047FFE780BD82
:1025700081B04FF080400068C007F0B1FFE74AF239
:102580000000C4F20A000068800700280AD5FFE7AF
:1025900040F20801C2F2000145F60020C0F26220BC
:1025A000086009E040F20801C2F2000142F6005062
:1025B000C0F231100860FFE788E04FF0804000680B
:1025C000C0F382000146009104286FD80099DFE82B
:1025D00001F0030B4048520040F20801C2F2000132
:1025E0004FF4FA40086061E04AF24000C4F20A0089
:1025F0000068800700280AD5FFE740F20801C2F210
:10260000000142F60050C0F23110086009E040F2CB
:102610000801C2F2000141F60030C0F2B7000860C4
:10262000FFE740F20801C2F2000108684AF6AB2257
:10263000CAF6AA22A0FB020250080001A0EB520039
:1026400082004FF6FE70C1F6FF7000EA520008608B
:102650002CE040F20801C2F200014FF40040086093
:1026600024E040F20801C2F2000141F60030C0F25D
:10267000B70008601AE040F20801C2F2000142F619
:102680000050C0F2311008604AF20000C4F20A00A3
:1026900000688007002808D5FFE740F20801C2F271
:1026A0000001086840000860FFE7FFE74FF0804046
:1026B00000688007002808D5FFE740F20801C2F251
:1026C00000010868C0080860FFE7FFE740F2080063
:1026D000C2F2000000684DF68361C4F21B31A0FB1A
:1026E0000110800C40F20401C2F20001086001B048
:1026F0007047000080B50821C4F20001086840F06E
:10270000007008609620FFF74BF8002000F0E2FD13
:10271000FFF72EFF40F20800C2F20000006840F60A
:102720000161C0F22771884204D3FFE79620FFF7CA
:1027300037F836E040F20800C2F2000000684BF2C1
:102740000141C0F2C441884204D3FFE77820FFF77B
:1027500027F825E040F20800C2F20000006845F6C4
:102760000121C0F26221884204D3FFE75020FFF725
:1027700017F814E040F20800C2F2000000684CF2C2
:102780008131C0F2C911884204D3FFE72820FFF746
:1027900007F803E01E20FFF703F8FFE7FFE7FFE776
:1027A000FFE740F28021C4F20A01086820F002002D
:1027B000086040F28011C4F20A01086820F00C00A1
:1027C00008607021C4F20001086820F0060008606B
:1027D000086840F00200086080BD000080B584B049
:1027E000029001208DF807000298008801460091B0
:1027F00040B1FFE700982C281FD0FFE70098312850
:1028000041D04EE0FFE741F2DC00C2F200004FF49D
:10281000617100F0A3FD41F60000C4F2040009213B
:10282000FFF792F941F29C11C2F200010120086009
:10283000FFE702992C200880FFE741F2DC00C2F29A
:10284000000000F077FD20B9FFE700208DF80F00B1
:1028500030E0FFE741F2DC00C2F20000642100F04A
:102860007DFD41F60000C4F204000921FFF74EF897
:1028700041F29C11C2F2000100200860FFE70299BA
:1028800031200880FFE741F2DC00C2F2000000F0D6
:1028900051FD20B9FFE700208DF80F000AE0FFE7A7
:1028A000B1E700208DF807000299088003208DF819
:1028B0000F00FFE79DF80F0004B080BD80B582B027
:1028C00000200190FFE741F2D400C2F2000000684E
:1028D00018B9FFE700F022FC5BE000200190FFE761
:1028E000019802284ED8FFE7019800EB800140F2E2
:1028F0000C00C2F2000010F8210008B9FFE73DE02B
:1029000041F2D400C2F200000368019800EB80019C
:1029100040F20C00C2F2000000EB81025168C91ABB
:102920005160019901EB810100EB810040680028B2
:1029300023DCFFE7019800EB800140F20C00C2F2BB
:10294000000000EB810251689368194451600199BD
:1029500001EB810100EB8100C06868B1FFE70198DD
:1029600000EB800140F20C00C2F2000000EB81009D
:10297000C16810308847FFE7FFE7FFE701980130A3
:102980000190ADE741F2D401C2F2000100200860DD
:10299000FFE798E780B584B0039041F2E400C2F20B
:1029A0000000029000208DF80700FFE79DF8070067
:1029B00004283FDCFFE70298007808B9FFE730E021
:1029C0000299086901380861002829DCFFE70298AC
:1029D000007A0146009140B1FFE70098012812D02B
:1029E000FFE70098022804D015E002990020087043
:1029F00015E00299CA6808691044086102984169A3
:102A0000806988470BE002990020087002984169AC
:102A10008069884703E0029900200870FFE7FFE71C
:102A2000FFE79DF8070001308DF8070002981C3081
:102A30000290BBE7002004B080BD000080B582B0EA
:102A4000019040F60000C4F20A0000F049F80020AE
:102A500002B080BD40F28002C2F20002D2E9000161
:102A6000013041F10001C2E9000141F2D401C2F29A
:102A700000010868013008607047000010B585B09B
:102A800004900391049B039C53E8001F890103D227
:102A9000BFF32F8F002204E043E8004000B1F3E7CA
:102AA0000122009202910190009805B010BD000033
:102AB00080B541F2D800C2F20000002100F054F9C4
:102AC00080BD000080B582B00190019941F64020A0
:102AD000C2F20000183000F037F902B080BD0000EB
:102AE00081B0009000995520086101B07047000046
:102AF00080B584B00390029101920821C4F20001D4
:102B0000086840F480600860039800F047F8039973
:102B1000886820F4706088600399886840F4806059
:102B20008860029848B9FFE70399886820F004009C
:102B30008860072000F058F80EE00399886840F09C
:102B40000400886002980399486003990120C860D6
:102B5000072000F07DF8FFE7019848B9FFE70399E7
:102B6000886820F00200886002980399086008E0F5
:102B70000399886840F00200886001980399086012
:102B8000FFE704B080BD000081B000900099886824
:102B900040F00100886001B07047000081B00090F3
:102BA0000099886820F00100886001B0704700003B
:102BB00081B08DF803009DF90300002812D4FFE7CF
:102BC0009DF9031001F01F02012090404A094EF2C6
:102BD0008011CEF2000141F82200BFF34F8FBFF306
:102BE0006F8FFFE701B0704781B08DF803009DF94A
:102BF0000300002812D4FFE79DF9031001F01F0223
:102C0000012090404A094EF28011CEF2000141F8B5
:102C10002200BFF34F8FBFF36F8FFFE701B0704704
:102C200081B08DF803009DF9030000280ED4FFE762
:102C30009DF9031001F01F02012090404A094EF255
:102C40000011CEF2000141F82200FFE701B0704709
:102C500081B08DF803009DF9030000280ED4FFE732
:102C60009DF9031001F01F02012090404A094EF225
:102C70000011CEF2000141F82200FFE701B07047D9
:102C800081B08DF803009DF9030000280ED4FFE702
:102C90009DF9031001F01F02012090404A094EF2F5
:102CA0000011CEF2000141F82200FFE701B07047A9
:102CB00082B08DF8070000919DF9070000280AD422
:102CC000FFE7009840019DF907104EF20042CEF256
:102CD000000288540BE0009840019DF8071001F0B5
:102CE0000F014EF61452CEF200028854FFE702B0F4
:102CF0007047000080B5012000F028FA80BD000078
:102D00007047000084B00390039B53E8002F511CD0
:102D100043E8001000B1F8E700920291019000989A
:102D200004B0704784B00390039BD3E84F2F511C2D
:102D3000C3E8401F00B1F8E78DF80320029101902D
:102D40009DF8030004B0704784B003900291039A89
:102D5000029B52E8001F42E8003000B1F9E7009101
:102D60000190009804B0704784B003908DF80B1068
:102D7000039A9DF80B30D2E84F1FC2E8403F00B1E4
:102D8000F9E78DF8031001909DF8030004B0704737
:102D900081B04EF21400CEF2000000684EF218012D
:102DA000CEF200010968401A00904EF60450CEF2AF
:102DB000000000684001002815D5FFE74EF214001E
:102DC000CEF2000000680099401A10280ADBFFE7E5
:102DD0004EF21400CEF20000006800990844013061
:102DE0000090FFE7FFE7009801B0704784B00390C0
:102DF00002914FF6FF70ADF80600FFE7029890B31E
:102E0000FFE70398411C03910178BDF8060080EAB2
:102E10000120ADF8060008200090FFE70098F0B10F
:102E2000FFE7BDF80600000400280DD5FFE7BDF858
:102E300006004000ADF80600BDF8060041F2210191
:102E40004840ADF8060005E0BDF806004000ADF8CA
:102E50000600FFE7FFE7009801380090DEE70298E0
:102E600001380290CAE7BDF8060004B070470000C0
:102E700081B04FF080400068C00710BBFFE74FF003
:102E80008040006800F01C010020B0EB910F0AD0D8
:102E9000FFE74FF08040006800F01C010220B0EB1B
:102EA000910F0ED1FFE700200090FFE70098132854
:102EB00006D8FFE700BFFFE7009801300090F5E774
:102EC0000FE000200090FFE7009844F61F61884261
:102ED00006D8FFE700BFFFE7009801300090F3E756
:102EE000FFE701B07047000080B586B005900598F7
:102EF00040F24C01C2F20001096880FB010103911C
:102F0000029041F29810C2F2000000685B2807DBD3
:102F1000FFE741F29810C2F200000068009002E062
:102F20005A200090FFE700980190029B0399019AB4
:102F3000D017D21A884101DBFFE71DE0019A029900
:102F40000398891A60EBE2700291039000F0B4F8E4
:102F500003460A4602990398C9185041029103900A
:102F6000FFE700F0A9F80246029B0398D21A71EB22
:102F7000000001DAFFE7F4E706B080BD80B586B057
:102F80000590059840F25001C2F20001096880FBEB
:102F900001010391029041F29810C2F20000006812
:102FA0005B2807DBFFE741F29810C2F200000068DF
:102FB000009002E05A200090FFE700980190029BE9
:102FC0000399019AD017D21A884101DBFFE71DE06F
:102FD000019A02990398891A60EBE27002910390BA
:102FE00000F06AF803460A4602990398C91850414E
:102FF00002910390FFE700F05FF80246029B0398FE
:10300000D21A71EB000001DAFFE7F4E706B080BDE9
:1030100080B584B002900191019840F20001C2F2A3
:103020000001884205D1FFE7029800F005F90390FE
:1030300003E04FF0FF300390FFE7039804B080BD3A
:1030400080B58AB000200690EFF3108107910799B0
:103050000491EFF3108172B60891049903910399DA
:1030600005910290FFE70298011D029100BBFFE766
:1030700041F67420C2F2000000680190FFF788FE5C
:103080000146019841F67022C2F200021268114412
:1030900040F24C02C2F20002126891FBF2F10844C5
:1030A0000690FFE705980990099880F31088DAE701
:1030B00006980AB080BD000080B58AB00020059057
:1030C0000490EFF31081079107990291EFF31081BB
:1030D00072B6089102990191019903910090FFE75E
:1030E0000098011D0091A8B9FFE7FFF751FE0146C6
:1030F000C81741F66822C2F20002D2E90032C918AC
:10310000504104910590FFE703980990099880F3D6
:103110001088E5E7049805990AB080BD80B582B0B3
:1031200041F2A010C2F2000001900168013101607B
:103130000068C1174FF20022C2F605220123FDF7F5
:10314000B9F80198026002B080BD000080B588B077
:103150008DF81300EFF31080059005980290EFF3BF
:10316000108072B60690029801900198039000209A
:103170000090FFE70098011D0091C0B9FFE79DF89E
:103180001300C00728B9FFE74FF08070FFF7BCF9C4
:10319000FFE74EF60451CEF200014FF000700860D8
:1031A000FFE703980790079880F31088E2E700F0A4
:1031B000E3F841F66821C2F200010020C1E90000F5
:1031C00041F67421C2F20001086041F67821C2F292
:1031D00000010860FFF794FD08B080BD80B582B0A3
:1031E0008DF807009DF8070010B9FFE702B080BD19
:1031F0009DF8071043F63E70C0F2000000F0E0F9C1
:10320000FFE7C8200090FFF76FFE0098FFF76CFE05
:10321000F7E7000080B582B000200190FFF76AFA5E
:10322000FEF706FEFEF7AAFDFEF71CFE62B6FFE7FC
:10323000FFF744FBFCE7000080B584B0029041F644
:103240008820C2F200000068082804D3FFE74FF08E
:10325000FF3003902BE0029941F68820C2F2000073
:1032600003685A1C026041F68022C2F20002D15467
:103270000068082804D0FFE702980A2814D1FFE765
:1032800041F68820C2F200000190026841F68021D8
:10329000C2F200014FF60060C0F20200FDF7DAFF53
:1032A000019900200860FFE702980390FFE7039868
:1032B00004B080BD80B54AF20001C4F20A010120C9
:1032C0000860FFF7D5FD4FF08041086840F001002D
:1032D000086080BD80B582B00190FFF7EBFFFEF77C
:1032E00001FE0421C4F20001012008604FF080417A
:1032F000086820F01C000860086840F004000860BE
:10330000019838B1FFE74FF08041086840F00200B3
:10331000086006E04FF08041086820F00200086075
:10332000FFE74FF08041086820F00100086002B01C
:1033300080BD000080B584B00390FFF781FE02904D
:10334000029803990968401A01900199039842680C
:1033500000209142A8BF012004B080BD80B582B09A
:1033600001900091009801994860FFF769FE01996A
:10337000086002B080BD000080B588B040F208004F
:10338000C2F2000001684DF68362C4F21B32A1FB59
:103390000221890C40F25002C2F200021160006862
:1033A00044F6D351C1F26201A0FB0110800940F242
:1033B0004C01C2F200010860EFF3108005900598FF
:1033C0000390EFF3108072B6069003980290029873
:1033D000049000200190FFE70198011D0191D8B9E8
:1033E000FFE7FFF769FE41F29012C2F2000200927D
:1033F000C2E90001FFF760FE0099D1E90012401A0E
:1034000041F29811C2F200010860FFE704980790AA
:10341000079880F31088DFE708B080BD83B04EF2D4
:103420001400CEF20000006801300290029B41F6C9
:103430006822C2F20002D2E90001C01841F1000185
:10344000C2E90001FFE7029A41F67021C2F20001D1
:10345000086810440860086840F24C02C2F200029A
:10346000136890FBF3F00190019812680B6800FB61
:1034700012300860019A41F67421C2F20001086816
:1034800010440860FFE7FFE7029A41F67C21C2F290
:103490000001086810440860086840F25002C2F257
:1034A0000002136890FBF3F00090009812680B681C
:1034B00000FB12300860009A41F67821C2F2000148
:1034C000086810440860FFE703B0704780B540F219
:1034D0004800C2F20000006844F60001C4F2040192
:1034E000884208D1FFE744F60000C4F20000012141
:1034F000FEF72AFBFFE740F24800C2F20000006836
:1035000044F20001C4F20401884206D1FFE74FF003
:1035100040200321FEF718FBFFE780BD80B540F295
:103520004800C2F20000006844F60001C4F2040141
:10353000884208D1FFE744F60000C4F200000121F0
:10354000FEF7E4F9FFE740F24800C2F2000000682D
:1035500044F20001C4F20401884206D1FFE74FF0B3
:1035600040200321FEF7D2F9FFE780BD80B582B08D
:1035700000208DF80700FEF759FF8DF807009DF831
:10358000070002B080BD000080B582B08DF8070052
:10359000FFF79CFFFFF7C2FF9DF80700FEF752FF01
:1035A0000A20FFF7EBFC02B080BD000080B582B0BE
:1035B0008DF807009DF80700FEF744FF02B080BDBC
:1035C0000FB4054B10B503A9044A029800F0DAF8CD
:1035D00010BC5DF814FB000011300000000000205A
:1035E00002E008C8121F08C1002AFAD170477047CC
:1035F000002001E001C1121F002AFBD1704700002A
:103600002DE9FF5F82B00021DDE90430020DDDF815
:1036100040B0034318D044F61050A2F2FF324243A8
:103620001514119801281FD0A5EB0B00401C5FEA70
:10363000000A4FF000064E4FDFF83891B046504672
:1036400015D5CAF1000413E0119801244AA30128FA
:1036500001D16FEA0B010298119AC0E90031C0E96B
:10366000024206B0BDE8F09FCBF10000DFE7044660
:103670000021404A491842EB0450CDE9001012E005
:10368000E00707D032463B4640464946FDF742F840
:103690008046894632463B4610461946FDF73AF8C1
:1036A00006460F466410002CEAD1DDE90401DDE98D
:1036B0000023BAF1000F06DAFDF72CF842464B461C
:1036C000FDF728F805E0FCF75BFE42464B46FCF7A9
:1036D00057FE04460E460022284BFDF7A5F803D8F6
:1036E0004FF0FF30014607E00022254B20463146CF
:1036F000FCF769FFFDF780F8102409E0002C0ADBD5
:103700000A220023FCF7C1FE039B30321A55641EC7
:1037100050EA0102F2D1641C039AC4F1110314446B
:10372000119A012A03D0012208430DD10AE008436F
:1037300004D000204FF0110B119072E7A3EB0B05A2
:103740006D1E0DE05B4504DD4FF0000205F1010543
:1037500004E003DA4FF00002A5F10105002AECD0E5
:1037600002981199C0E90231C0E9004579E70000EB
:10377000000014400000F03F300000000000F04363
:103780000000E03F2DE9FF4F95B09B468946064675
:1037900000250FE2252877D100242746F84A012189
:1037A000059400E0044316F8013F203B01FA03F0C2
:1037B0001042F7D130782A2811D06FF02F033078DB
:1037C000A0F13002092A16D8059A44F0020402EB4F
:1037D000820203EB42021044761C0590EFE759F891
:1037E000042B0592002A03DA504244F40054059059
:1037F00044F00204761C30782E2816D116F8010FFA
:1038000044F004042A280DD06FF02F023078A0F184
:103810003003092B09D807EB870302EB4303C718D2
:10382000761CF3E759F8047B761C30786C280FD0AF
:1038300006DC4C2817D068280DD06A2814D104E083
:10384000742810D07A280FD10DE044F400140AE057
:1038500044F4801401E044F440147278824202D1AE
:1038600004F58014761C761C307866280BD013DCA7
:10387000582877D009DC002875D04528F6D046288E
:10388000F4D047281AD19DE118E0632835D0642888
:1038900079D0652812D195E1702873D008DC6728AB
:1038A000F1D069286FD06E280DD06F2806D1B5E011
:1038B00073282CD0752875D0782874D05A4617995B
:1038C00090476D1C75E1C4F30250022809D003280B
:1038D0000DD0D9F8001004280DD00D6009F10409AD
:1038E00067E1D9F80010EA17C1E90052F6E7D9F804
:1038F00000100D80F2E70D70F0E719F8041B8DF849
:10390000001000208DF80100EA46012003E059F87C
:1039100004AB4FF0FF3061074FF0000102D40DE01F
:1039200008F101018846B9420FDA8045F8DB1AF840
:1039300008100029F4D108E008F10101884681420D
:10394000FADB1AF808100029F6D105985B46A0EBBF
:10395000080721463846179A00F094FA284400EBED
:10396000080507E04DE029E10DE01AF8010B5A4681
:1039700017999047B8F10108F7D25B4621463846BF
:10398000179A13E142E00A220092C4F302524FF068
:10399000000A022A08D059F804CB032A4FEAEC7136
:1039A0000AD00DE029E02AE009F1070121F0070221
:1039B000F2E802C1914609E00FFA8CFC4FEAEC7183
:1039C000042A03D14FFA8CFC4FEAEC71002907DA84
:1039D0000A460021DCF1000C61EB02012D2202E01D
:1039E000220504D52B228DF80420012203E0E207F2
:1039F00001D02022F7E7904659E00A2102E0102288
:103A00000DE010214FF0000A00910BE010224FF062
:103A1000000A44F004040827009203E008224FF053
:103A2000000A0092C4F30252022A05D059F804CBCE
:103A30000021032A08D009E009F1070121F007025B
:103A4000F2E802C1914605E01FFA8CFC042A01D17C
:103A50000CF0FF0C4FF00008220728D5702806D084
:103A6000009B83F0100353EA0A0305D00EE04022C6
:103A70008DF80420012208E05CEA010206D0302221
:103A80008DF804208DF8050002229046009B83F0FB
:103A9000080353EA0A030AD15CEA010201D1620772
:103AA00005D530228DF804204FF001087F1E5828DC
:103AB00004D034A003900EA802900DE036A0F9E7E0
:103AC00053466046009AFCF7E0FC84460398825C0B
:103AD0000298401E029002705CEA0100F0D1029848
:103AE00006A9081A00F1200A600702D524F48034E0
:103AF00000E00127574502DDA7EB0A0000E00020A7
:103B000000EB0A01009005984144401A0590E0033B
:103B100006D45B462146179A059800F0B3F9054490
:103B2000002706E001A85A46C05D179990476D1C12
:103B30007F1C4745F6DBE0030CD55B462146179A10
:103B4000059800F09FF9054404E030205A46179983
:103B500090476D1C0099481E00900029F5DC08E094
:103B6000029802995A460078491C02911799904789
:103B70006D1CBAF10001AAF1010AF1DC65E1000057
:103B80000928010030313233343536373839616233
:103B900063646566000000003031323334353637F7
:103BA00038394142434445460000000000F058F9CE
:103BB0000544761C307800287FF4ECAD19B0284617
:103BC000BDE8F08F620700D4062709F1070222F052
:103BD000070CFCE80223E14603F000485FEA080C0A
:103BE00002D00FF2702C0DE05FEA045C02D50FF2F8
:103BF000682C07E05FEAC47C02D00FF2602C01E081
:103C0000AFF2700C4FF0FF3823F00043CDF850C0F6
:103C100065280CD006DC452809D046281DD0472849
:103C20003DD13DE0662818D067287ED138E00021DC
:103C3000112F01DB112000E0781CCDE9000106A95D
:103C40000EA8FFF7DDFCDDE90F010E9A03910021BC
:103C5000009207F1010A04914DE04FF000400097F7
:103C6000CDE9011006A90EA8FFF7CAFCDDE90F0295
:103C700003920E9B11990022DDF80CA00093049290
:103C800011B9791C00EB010AB7EB0A0004D4C0F1AA
:103C9000FF3007F1010A0490AAEB0700019044E00D
:103CA000012F00DA01270021112F01DD112000E092
:103CB0003846CDE9000106A90EA8FFF7A1FCDDE911
:103CC0000F010E9A0391002104910092BA46210738
:103CD0000CD40399514500DA8A46BAF1010F05DD8B
:103CE000009AAAF10101515C302908D0B84202DAE9
:103CF00010F1040F06DA0121CDE9011015E0AAF157
:103D00000101E9E7002805DC049901440491AAEBCC
:103D1000000102E0411C514500DD8A460499401A29
:103D2000401C01904FF000400290200704D40198FD
:103D3000504501DBCDF8048000208DF84F0002983B
:103D40000DF14F07B0F1004F25D02B200E900298B7
:103D50004FF0020800280CDA404202902D200E900D
:103D600007E00A210298FCF77AFB3031029007F84D
:103D7000011DB8F10001A8F10108F2DC0298002849
:103D8000EFD1791E0E980870307800F0200040F0D6
:103D9000450007F8020D12A8C01B00F1070814988F
:103DA000007800B1012000EB0A01019801EBE071FD
:103DB00005984144401A401E0590E00306D45B4636
:103DC0002146179A059800F05DF80544149800788C
:103DD00018B15A46179990476D1CE00324D55B46ED
:103DE0002146179A059800F04DF805441CE0049808
:103DF000002807DBDDE90301884203DD0098405C11
:103E0000179901E0179930205A469047049805F118
:103E10000105401C04900198401E019004D12E2001
:103E20005A46179990476D1CBAF10001AAF1010A90
:103E3000DDDC05E017F8010B5A46179990476D1C19
:103E4000B8F10001A8F10108F4DC5B462146179A9D
:103E50000598ABE62D0000002B00000020000000BC
:103E60002DE9F041044600251E461746880404D477
:103E700005E039462020B0476D1C641EF9D5284660
:103E8000BDE8F0812DE9F041044600251E4690462C
:103E9000C80301D5302700E02027880404D505E0B9
:103EA00041463846B0476D1C641EF9D52846BDE82A
:103EB000F08100000100010180000000C01100201D
:103EC000C0190020401A0020000000005461736BEC
:103ED0002053746172740D0A0053494E545F535459
:103EE00041545F444953434F4E4E454354200D0ABD
:103EF00000496E697420737461747573203A2047A9
:103F0000494E545F535441545F5048595F434841B0
:103F10004E47450D0A0053494E545F535441545F78
:103F2000434F4E4E4543540D0A0053494E545F5380
:103F30005441545F54494D5F4F55540D0A0045722A
:103F4000726F723A20253032580D0A00726563652F
:103F5000697665206C656E203D2025640D0A00435E
:103F60004833393245565420546573742044656D86
:103F70006F0D0A00434833393220436F6E6E65631C
:103F8000742045746865726E65740D0A00202020E7
:103F9000202532780D0A00434833393256455220E5
:103FA0003A202532780D0A004348333932496E6988
:103FB00074004348333932434D44496E6974434871
:103FC000333932004348333932434D4443686563E3
:103FD0006B45786973740000004000000000002009
:103FE00080000000E03500008040000080000020DC
:103FF000105A0000F0350000FDECFFFF000000004B
:10400000000000000C000000002D31010101000043
:104010000A0000000A0000009529000000000000CE
:10402000010101000A0000000A000000DD27000075
:104030000000000001010200F4010000F401000092
:104040003D2A00000000000000480440010000007C
:1040500001000000C0A83D648913E8FD0200E601EC
:10406000010188131192020000000000000000000E
:104070000000000000000000000000000000000040
:04000005000001A94D
:00000001FF
